Microchip MPLAB XC8 Compiler V2.32

Linker command line:

-W-3 --edf=/opt/microchip/xc8/v2.32/pic/dat/en_msgs.txt -cn \
  -h+dist/default/production/UART_RC_16F627.X.production.sym \
  --cmf=dist/default/production/UART_RC_16F627.X.production.cmf -z \
  -Q16F628A -o/tmp/xcXebJofA --defsym=__MPLAB_BUILD=1 \
  -Mdist/default/production/UART_RC_16F627.X.production.map -E1 \
  -ver=XC8 Compiler --acfsm=1493 -ASTACK=0BEh-0EFh -pstack=STACK \
  -ACODE=00h-07FFh -ASTRCODE=00h-07FFh -ASTRING=00h-0FFhx8 \
  -ACONST=00h-0FFhx8 -AENTRY=00h-0FFhx8 -ACOMMON=070h-07Fh \
  -ABANK0=020h-06Fh -ABANK1=0A0h-0EFh -ABANK2=0120h-014Fh \
  -ARAM=020h-06Fh,0A0h-0EFh,0120h-014Fh \
  -AABS1=020h-07Fh,0A0h-0EFh,0120h-014Fh -ASFR0=00h-01Fh -ASFR1=080h-09Fh \
  -ASFR2=0100h-011Fh -ASFR3=0180h-01EFh -ACONFIG=02007h-02007h -DCONFIG=2 \
  -AIDLOC=02000h-02003h -DIDLOC=2 -AEEDATA=00h-07Fh/02100h \
  -peeprom_data=EEDATA -DEEDATA=2 -DCODE=2 -DSTRCODE=2 -DSTRING=2 -DCONST=2 \
  -DENTRY=2 -preset_vec=00h,intentry,init,end_init -ppowerup=CODE \
  -pcinit=CODE -pfunctab=ENTRY -k /tmp/xcXegmGpb.o \
  dist/default/production/UART_RC_16F627.X.production.o 

Object code version is 3.11

Machine type is 16F628A



                Name                               Link     Load   Length Selector   Space Scale
/tmp/xcXegmGpb.o
                end_init                              0        0        1        0       0
                config                             2007     2007        1        0       4
dist/default/production/UART_RC_16F627.X.production.o
                cinit                               7CD      7CD       33      F9A       0
                config                             2007     2007        1        0       4
                text16                              3C1      3C1        8      782       0
                text15                              3E7      3E7       12      7CE       0
                text14                              3D1      3D1        A      7A2       0
                text13                              5CE      5CE       68      B9C       0
                text12                              51E      51E       54      A3C       0
                text11                              493      493       45      926       0
                text10                              636      636       75      C6C       0
                text9                               3DB      3DB        C      7B6       0
                text8                               474      474       1F      8E8       0
                text7                               4D8      4D8       46      9B0       0
                text6                               3F9      3F9       12      7F2       0
                text5                               444      444       18      888       0
                text4                               40B      40B       12      816       0
                text3                               45C      45C       18      8B8       0
                text2                               41D      41D       13      83A       0
                text1                               6AB      6AB      122      D56       0
                maintext                            572      572       5C      AE4       0
                cstackBANK0                          20       20       1C       20       1
                cstackCOMMON                         70       70        E       70       1
                clrtext                             3C9      3C9        8      792       0
                bssBANK1                             A0       A0       1E       A0       1
                dataBANK0                            55       55       14       20       1
                bssBANK0                             3C       3C       19       20       1
                idataBANK0                          430      430       14      860       0

TOTAL           Name                               Link     Load   Length     Space
        CLASS   STACK          

        CLASS   CODE           
                end_init                              0        0        1         0
                cinit                               7CD      7CD       33         0
                text16                              3C1      3C1        8         0
                text15                              3E7      3E7       12         0
                text14                              3D1      3D1        A         0
                text13                              5CE      5CE       68         0
                text12                              51E      51E       54         0
                text11                              493      493       45         0
                text10                              636      636       75         0
                text9                               3DB      3DB        C         0
                text8                               474      474       1F         0
                text7                               4D8      4D8       46         0
                text6                               3F9      3F9       12         0
                text5                               444      444       18         0
                text4                               40B      40B       12         0
                text3                               45C      45C       18         0
                text2                               41D      41D       13         0
                text1                               6AB      6AB      122         0
                maintext                            572      572       5C         0
                clrtext                             3C9      3C9        8         0
                idataBANK0                          430      430       14         0

        CLASS   STRCODE        

        CLASS   STRING         

        CLASS   CONST          

        CLASS   ENTRY          

        CLASS   COMMON         
                cstackCOMMON                         70       70        E         1

        CLASS   BANK0          
                cstackBANK0                          20       20       1C         1
                dataBANK0                            55       55       14         1
                bssBANK0                             3C       3C       19         1

        CLASS   BANK1          
                bssBANK1                             A0       A0       1E         1

        CLASS   BANK2          

        CLASS   RAM            

        CLASS   ABS1           
                abs_s1                               7E       7E        2         1

        CLASS   SFR0           

        CLASS   SFR1           

        CLASS   SFR2           

        CLASS   SFR3           

        CLASS   CONFIG         
                config                             2007     2007        1         4

        CLASS   IDLOC          

        CLASS   EEDATA         

        CLASS   BANK3          



SEGMENTS        Name                           Load    Length   Top    Selector   Space  Class     Delta

                text15                         0003E7  000012  0003F9       7CE       0  CODE        2
                text9                          0003DB  00000C  0003E7       7B6       0  CODE        2
                text6                          0003F9  000012  00040B       7F2       0  CODE        2
                text5                          000444  000018  00045C       888       0  CODE        2
                text3                          00045C  000018  000474       8B8       0  CODE        2
                text8                          000474  00001F  000493       8E8       0  CODE        2
                text4                          00040B  000012  00041D       816       0  CODE        2
                text2                          00041D  000013  000430       83A       0  CODE        2
                idataBANK0                     000430  000014  000444       860       0  CODE        2
                text16                         0003C1  000008  0003C9       782       0  CODE        2
                reset_vec                      000000  000001  000001         0       0  CODE        2
                clrtext                        0003C9  000008  0003D1       792       0  CODE        2
                text14                         0003D1  00000A  0003DB       7A2       0  CODE        2
                cstackBANK0                    000020  000049  000069        20       1  BANK0       1
                text1                          0006AB  000122  0007CD       D56       0  CODE        2
                cinit                          0007CD  000033  000800       F9A       0  CODE        2
                cstackCOMMON                   000070  00000E  00007E        70       1  COMMON      1
                bssBANK1                       0000A0  00001E  0000BE        A0       1  BANK1       1
                text12                         00051E  000054  000572       A3C       0  CODE        2
                text7                          0004D8  000046  00051E       9B0       0  CODE        2
                text11                         000493  000045  0004D8       926       0  CODE        2
                text10                         000636  000075  0006AB       C6C       0  CODE        2
                text13                         0005CE  000068  000636       B9C       0  CODE        2
                maintext                       000572  00005C  0005CE       AE4       0  CODE        2


UNUSED ADDRESS RANGES

        Name                Unused          Largest block    Delta
        BANK0            0069-006F              7           1
        BANK1            00BE-00EF             32           1
        BANK2            0120-014F             30           1
        CODE             0001-03C0            3C0           2
        CONST            0001-03C0            100           2
        EEDATA           2100-217F             80           2
        ENTRY            0001-03C0            100           2
        IDLOC            2000-2003              4           2
        RAM              0069-006F              7           1
                         00BE-00EF             32
                         0120-014F             30
        SFR0             0000-001F             20           1
        SFR1             0080-009F             20           1
        SFR2             0100-011F             20           1
        SFR3             0180-01EF             70           1
        STACK            00BE-00EF             32           1
        STRCODE          0001-03C0            3C0           2
        STRING           0001-03C0            100           2

                                  Symbol Table

?___lldiv                cstackBANK0  0020
?___llmod                cstackCOMMON 0070
?___lmul                 cstackCOMMON 0070
?_strtol                 cstackBANK0  0020
_BRGH                    (abs)        04C2
_CMCON                   (abs)        001F
_CREN                    (abs)        00C4
_INTCONbits              (abs)        000B
_PORTAbits               (abs)        0005
_PORTB                   (abs)        0006
_RCIE                    (abs)        0465
_RCIF                    (abs)        0065
_RCREG                   (abs)        001A
_SPBRG                   (abs)        0099
_SPEN                    (abs)        00C7
_SYNC                    (abs)        04C4
_TRISA                   (abs)        0085
_TRISB                   (abs)        0086
_TRISBbits               (abs)        0086
__Habs1                  abs1         0000
__Hbank0                 bank0        0000
__Hbank1                 bank1        0000
__Hbank2                 bank2        0000
__Hbank3                 bank3        0000
__HbssBANK0              bssBANK0     0000
__HbssBANK1              bssBANK1     0000
__Hcinit                 cinit        0800
__Hclrtext               clrtext      0000
__Hcode                  code         0000
__Hcommon                common       0000
__Hconfig                config       2008
__HcstackBANK0           cstackBANK0  0000
__HcstackCOMMON          cstackCOMMON 0000
__HdataBANK0             dataBANK0    0000
__Heeprom_data           eeprom_data  0000
__Hend_init              end_init     0001
__Hfunctab               functab      0000
__HidataBANK0            idataBANK0   0000
__Hinit                  init         0000
__Hintentry              intentry     0000
__Hmaintext              maintext     0000
__Hpowerup               powerup      0000
__Hram                   ram          0000
__Hreset_vec             reset_vec    0000
__Hsfr0                  sfr0         0000
__Hsfr1                  sfr1         0000
__Hsfr2                  sfr2         0000
__Hsfr3                  sfr3         0000
__Hspace_0               (abs)        0800
__Hspace_1               (abs)        00BE
__Hspace_2               (abs)        0000
__Hspace_3               (abs)        0000
__Hspace_4               (abs)        400F
__Hstack                 stack        0000
__Hstrings               strings      0000
__Htext                  text         0000
__Labs1                  abs1         0000
__Lbank0                 bank0        0000
__Lbank1                 bank1        0000
__Lbank2                 bank2        0000
__Lbank3                 bank3        0000
__LbssBANK0              bssBANK0     0000
__LbssBANK1              bssBANK1     0000
__Lcinit                 cinit        07CD
__Lclrtext               clrtext      0000
__Lcode                  code         0000
__Lcommon                common       0000
__Lconfig                config       0000
__LcstackBANK0           cstackBANK0  0000
__LcstackCOMMON          cstackCOMMON 0000
__LdataBANK0             dataBANK0    0000
__Leeprom_data           eeprom_data  0000
__Lend_init              end_init     0000
__Lfunctab               functab      0000
__LidataBANK0            idataBANK0   0000
__Linit                  init         0000
__Lintentry              intentry     0000
__Lmaintext              maintext     0000
__Lpowerup               powerup      0000
__Lram                   ram          0000
__Lreset_vec             reset_vec    0000
__Lsfr0                  sfr0         0000
__Lsfr1                  sfr1         0000
__Lsfr2                  sfr2         0000
__Lsfr3                  sfr3         0000
__Lspace_0               (abs)        0000
__Lspace_1               (abs)        0000
__Lspace_2               (abs)        0000
__Lspace_3               (abs)        0000
__Lspace_4               (abs)        0000
__Lstack                 stack        0000
__Lstrings               strings      0000
__Ltext                  text         0000
__S0                     (abs)        0800
__S1                     (abs)        00BE
__S2                     (abs)        0000
__S3                     (abs)        0000
___int_sp                stack        0000
___latbits               (abs)        0000
___lldiv                 text13       05CE
___lldiv@counter         cstackBANK0  002C
___lldiv@dividend        cstackBANK0  0024
___lldiv@divisor         cstackBANK0  0020
___lldiv@quotient        cstackBANK0  0028
___llmod                 text12       051E
___llmod@counter         cstackCOMMON 0079
___llmod@dividend        cstackCOMMON 0074
___llmod@divisor         cstackCOMMON 0070
___lmul                  text7        04D8
___lmul@multiplicand     cstackCOMMON 0074
___lmul@multiplier       cstackCOMMON 0070
___lmul@product          cstackCOMMON 0079
___sp                    stack        0000
___stackhi               (abs)        0000
___stacklo               (abs)        0000
__end_of___lldiv         text13       0636
__end_of___llmod         text12       0572
__end_of___lmul          text7        051E
__end_of__initialization cinit        07FE
__end_of_bootPic         text16       03C9
__end_of_initRcUART      text15       03F9
__end_of_isalpha         text5        045C
__end_of_isdigit         text4        041D
__end_of_isspace         text3        0474
__end_of_isupper         text6        040B
__end_of_main            maintext     05CE
__end_of_muxInit         text14       03DB
__end_of_muxNumber       text10       06AB
__end_of_muxView         text11       04D8
__end_of_rcRead          text9        03E7
__end_of_rcReadString    text8        0493
__end_of_strtol          text1        07CD
__end_of_toupper         text2        0430
__initialization         cinit        07CD
__pbssBANK0              bssBANK0     003C
__pbssBANK1              bssBANK1     00A0
__pcstackBANK0           cstackBANK0  0020
__pcstackCOMMON          cstackCOMMON 0070
__pdataBANK0             dataBANK0    0055
__pidataBANK0            idataBANK0   0430
__pmaintext              maintext     0572
__ptext1                 text1        06AB
__ptext10                text10       0636
__ptext11                text11       0493
__ptext12                text12       051E
__ptext13                text13       05CE
__ptext14                text14       03D1
__ptext15                text15       03E7
__ptext16                text16       03C1
__ptext2                 text2        041D
__ptext3                 text3        045C
__ptext4                 text4        040B
__ptext5                 text5        0444
__ptext6                 text6        03F9
__ptext7                 text7        04D8
__ptext8                 text8        0474
__ptext9                 text9        03DB
__size_of___lldiv        (abs)        0000
__size_of___llmod        (abs)        0000
__size_of___lmul         (abs)        0000
__size_of_bootPic        (abs)        0000
__size_of_initRcUART     (abs)        0000
__size_of_isalpha        (abs)        0000
__size_of_isdigit        (abs)        0000
__size_of_isspace        (abs)        0000
__size_of_isupper        (abs)        0000
__size_of_main           (abs)        0000
__size_of_muxInit        (abs)        0000
__size_of_muxNumber      (abs)        0000
__size_of_muxView        (abs)        0000
__size_of_rcRead         (abs)        0000
__size_of_rcReadString   (abs)        0000
__size_of_strtol         (abs)        0000
__size_of_toupper        (abs)        0000
_bootPic                 text16       03C1
_dataNum                 bssBANK0     0040
_dataRc                  bssBANK1     00A0
_dataRc_c                bssBANK0     0054
_dec                     bssBANK0     004C
_initRcUART              text15       03E7
_isalpha                 text5        0444
_isalpha$631             cstackCOMMON 0072
_isdigit                 text4        040B
_isdigit$634             cstackCOMMON 0070
_isspace                 text3        045C
_isspace$637             cstackCOMMON 0070
_isupper                 text6        03F9
_isupper$640             cstackCOMMON 0070
_main                    maintext     0572
_muxInit                 text14       03D1
_muxNumber               text10       0636
_muxView                 text11       0493
_numbers                 dataBANK0    0055
_rcRead                  text9        03DB
_rcReadString            text8        0474
_strtol                  text1        06AB
_toupper                 text2        041D
_uni                     bssBANK0     0050
btemp                    (abs)        007E
clear_ram0               clrtext      03C9
end_of_initialization    cinit        07FE
intlevel0                functab      0000
intlevel1                functab      0000
intlevel2                functab      0000
intlevel3                functab      0000
intlevel4                functab      0000
intlevel5                functab      0000
isalpha@c                cstackCOMMON 0073
isdigit@c                cstackCOMMON 0071
isspace@c                cstackCOMMON 0071
isupper@c                cstackCOMMON 0071
main@cont                cstackBANK0  0037
main@ref                 cstackBANK0  003B
muxNumber@num            cstackBANK0  002D
muxNumber@numDigits      cstackBANK0  0031
muxNumber@res            bssBANK0     0048
muxView@digitsView       cstackCOMMON 0070
rcReadString@i           cstackCOMMON 0076
rcReadString@out         cstackCOMMON 0075
rcReadString@size        cstackCOMMON 0071
reset_vec                reset_vec    0000
start                    init         0000
start_initialization     cinit        07CD
strtol@a                 cstackBANK0  0029
strtol@base              cstackBANK0  0021
strtol@c                 cstackBANK0  002E
strtol@endptr            cstackBANK0  0020
strtol@s                 cstackBANK0  002D
strtol@sign              cstackBANK0  0028
toupper@c                cstackCOMMON 0071
wtemp0                   (abs)        007E


MODULE INFORMATION

Module		Function		Class		Link	Load	Size
/opt/microchip/xc8/v2.32/pic/sources/c90/common/__lldiv.c
		___lldiv       		CODE           	05CE	0000	104

/opt/microchip/xc8/v2.32/pic/sources/c90/common/__lldiv.c estimated size: 104

/opt/microchip/xc8/v2.32/pic/sources/c90/common/strtol.c
		_strtol        		CODE           	06AB	0000	290

/opt/microchip/xc8/v2.32/pic/sources/c90/common/strtol.c estimated size: 290

/opt/microchip/xc8/v2.32/pic/sources/c90/common/isalpha.c
		_isalpha       		CODE           	0444	0000	24

/opt/microchip/xc8/v2.32/pic/sources/c90/common/isalpha.c estimated size: 24

mainRc.c
		_bootPic       		CODE           	03C1	0000	8
		_main          		CODE           	0572	0000	92
		_initRcUART    		CODE           	03E7	0000	18
		_rcRead        		CODE           	03DB	0000	12
		_rcReadString  		CODE           	0474	0000	31

mainRc.c estimated size: 161

/opt/microchip/xc8/v2.32/pic/sources/c90/common/isdigit.c
		_isdigit       		CODE           	040B	0000	18

/opt/microchip/xc8/v2.32/pic/sources/c90/common/isdigit.c estimated size: 18

./dispMux.c
		_muxInit       		CODE           	03D1	0000	10
		_muxNumber     		CODE           	0636	0000	117
		_muxView       		CODE           	0493	0000	69

./dispMux.c estimated size: 196

shared
		__initialization		CODE           	07CD	0000	49

shared estimated size: 49

/opt/microchip/xc8/v2.32/pic/sources/c90/common/Umul32.c
		___lmul        		CODE           	04D8	0000	70

/opt/microchip/xc8/v2.32/pic/sources/c90/common/Umul32.c estimated size: 70

/opt/microchip/xc8/v2.32/pic/sources/c90/common/llmod.c
		___llmod       		CODE           	051E	0000	84

/opt/microchip/xc8/v2.32/pic/sources/c90/common/llmod.c estimated size: 84

/opt/microchip/xc8/v2.32/pic/sources/c90/common/isupper.c
		_isupper       		CODE           	03F9	0000	18

/opt/microchip/xc8/v2.32/pic/sources/c90/common/isupper.c estimated size: 18

/opt/microchip/xc8/v2.32/pic/sources/c90/common/toupper.c
		_toupper       		CODE           	041D	0000	19

/opt/microchip/xc8/v2.32/pic/sources/c90/common/toupper.c estimated size: 19

/opt/microchip/xc8/v2.32/pic/sources/c90/common/isspace.c
		_isspace       		CODE           	045C	0000	24

/opt/microchip/xc8/v2.32/pic/sources/c90/common/isspace.c estimated size: 24

